:1000000012C03FC018951895189518951895189511
:100010001895189518951895189518951895189578
:100020001895189518958FE58DBFC0E4E8E34E2E1E
:1000300084E08EBFD4E0F4E05F2EEEEFF3E0A0E6C4
:10004000B0E088278D933197E9F766248D9A8E9AD0
:100050008A9885B7836085BF78948BB780648BBF9F
:10006000959A88EE93E054D0959888EE93E050D01E
:10007000969A88EE93E04CD0969888EE93E048D01C
:10008000EFCF0F921F922F923F924F925F927F92EB
:10009000AF92BF920F931F932F933F934F935F9312
:1000A0006F937F938F939F93AF93BF93CF93DF9380
:1000B000EF93FF938FB78F93959A969A84EF91E081
:1000C00027D0959896988F918FBFFF91EF91DF91F0
:1000D000CF91BF91AF919F918F917F916F915F91E0
:1000E0004F913F912F911F910F91BF90AF907F90B3
:1000F0005F904F903F902F901F900F9018953197E1
:10010000F1F70895689462F80895E89462F8089504
:10011000EF93FF93EE27E82BE92B31F0EAEFF0E0C5
:0E0120003197F1F70197D1F7FF91EF91089514
:00000001FF
